:020000040000FA
:100000000C94C3010C94EB010C94EB010C94EB01E8
:100010000C94EB010C94EB010C94EB010C94EB01B0
:100020000C94EB010C94EB010C94EB010C94EB01A0
:100030000C94EB010C94EB010C94EB010C94EB0190
:100040000C94381A0C94EB010C94061A0C94E019D9
:100050000C94EB010C94EB010C94EB010C94EB0170
:100060000C94821A0C94EB01084AD73B3BCE016EEC
:1000700084BCBFFDC12F3D6C74319ABD56833DDAFF
:100080003D00C77F11BED9E4BB4C3E916BAAAABE0E
:10009000000000803F07634236B79BD8A71A396833
:1000A0005618AEBAAB558C1D3CB7CC5763BD6DED41
:1000B000FD753EF6177231BF000000803F0800005A
:1000C00000BE922449123EABAAAA2ABECDCCCC4C8B
:1000D0003E00000080BEABAAAAAA3E00000000BFFE
:1000E000000000803F0000000000084178D3BB43BF
:1000F00087D1133D190E3CC3BD4282AD2B3E68EC47
:100100008276BED98FE1A93E4C80EFFFBE01C4FFCD
:100110007F3F0000000000004E414E494E495459B7
:10012000494E46CDCCCC3D0AD7233C17B7D13877C2
:10013000CC2B329595E6241FB14F0A0000204100D8
:1001400000C84200401C4620BCBE4CCA1B0E5AAE22
:10015000C59D7400407A10F35A00A0724E18090031
:1001600010A5D4E80000E87648170000E40B54021C
:100170000000CA9A3B000000E1F505000080969857
:1001800000000040420F000000A0860100000010A7
:100190002700000000E803000000006400000000E9
:1001A000000A00000000000100000000002C76D8CA
:1001B00088DC674F0823DFC1DFAE59E1B1B796E5B0
:1001C000E3E453C63AE651997696E8E6C28426EB14
:1001D000898C9B62ED407C6FFCEFBC9C9F40F2BA27
:1001E000A56FA5F490055A2AF75C936B6CF9676DBF
:1001F000C11BFCE0E40D47FEF520E6B500D0ED9014
:100200002E0300943577050080841E080000204EE0
:100210000A000000C80C333333330F986E12831179
:1002200041EF8D2114893BE65516CFFEE6DB18D150
:10023000844B381BF77C1D901DA4BBE42420328422
:10024000725E228100C9F124ECA1E53D273E6128C0
:10025000782C792C7A292F673A00543D0049522096
:10026000466C616D65204C6576656C3D0047617339
:10027000206C6576656C3D0023496E76616C69641F
:10028000206B65792100482D6669656C643A2028E9
:100290000000000000240027002A000000000025C4
:1002A0000028002B0023626D70206661696C656414
:1002B000002357656C636F6D6520746F20757365DF
:1002C000204E616E6F204C6F67676572004D533D25
:1002D00000234E6F2055562073656E736F72210098
:1002E000503D0042543D004448543D002344757243
:1002F0006174696F6E3D0054494D45443D0023498A
:100300006E74657276616C3D0054494D45493D00FF
:1003100053484F57533D004C6F67676572204E61DD
:100320006D653A20004C4F474745520056455253A1
:10033000494F4E005245424F4F54000000000023E9
:100340000026002900040404040404040402020238
:100350000202020303030303030102040810204006
:10036000800102040810200102040810200000008F
:100370000800020100000304070000000000000064
:100380000000A11BD22211241FBECFEFD8E0DEBF98
:10039000CDBF12E0A0E0B1E0ECEEFDE502C00590BB
:1003A0000D92A631B107D9F724E0A6E1B2E001C071
:1003B0001D92A036B207E1F711E0C2ECD1E004C013
:1003C0002197FE010E94CC2CC13CD107C9F70E94A5
:1003D000871C0C94E92E0C94000090919802809157
:1003E00097022FEF3FEF981748F4E92FF0E0E95814
:1003F000FD4F208130E09F5F90939802C9010895DE
:1004000090919802809197022FEF3FEF981748F450
:10041000E92FF0E0E958FD4F208130E09F5F909395
:100420009802C901089591E09093C5028093E70274
:100430001092C6021092E802089508950895089552
:10044000AF92BF92CF92DF92EF92FF920F931F93E2
:10045000CF93DF936C017B018B01040F151FEB0120
:100460005E01AE18BF08C017D10759F06991D601D7
:10047000ED91FC910190F081E02DC6010995892B49
:1004800079F7C501DF91CF911F910F91FF90EF9008
:10049000DF90CF90BF90AF900895CF93DF93FC0192
:1004A000448155816081718189EE92E00E94200231
:1004B000EC0142E050E066E471E089EE92E00E94D7
:1004C00020028C0F9D1FDF91CF910895FC01538D69
:1004D000448D252F30E0842F90E0821B930B54171E
:1004E00010F0CF96089501970895FC01918D828DAB
:1004F000981761F0A28DAE0FBF2FB11D5D968C9144
:10050000928D9F5F9F73928F90E008958FEF9FEF82
:100510000895FC01918D828D981731F0828DE80F3E
:10052000F11D858D90E008958FEF9FEF0895FC01F8
:10053000918D228D892F90E0805C9F4F821B9109C5
:100540008F739927089589EE92E00E94970221E027
:10055000892B09F420E0822F089580E090E0892B18
:1005600029F00E94A30281110C9400000895FC015F
:10057000A48DA80FB92FB11DA35ABF4F2C91848D04
:1005800090E001968F739927848FA689B7892C9361
:10059000A089B1898C91837080648C93938D848DB4
:1005A000981306C00288F389E02D80818F7D8083B7
:1005B0000895EF92FF920F931F93CF93DF93EC0177
:1005C00081E0888F9B8D8C8D98131AC0E889F989FA
:1005D000808185FF15C09FB7F894EE89FF896083FD
:1005E000E889F98980818370806480839FBF81E07E
:1005F00090E0DF91CF911F910F91FF90EF900895C0
:10060000F62E0B8D10E00F5F1F4F0F731127E02E9A
:100610008C8D8E110CC00FB607FCFACFE889F989D2
:10062000808185FFF5CFCE010E94B702F1CFEB8D1F
:10063000EC0FFD2FF11DE35AFF4FF0829FB7F894A6
:100640000B8FEA89FB8980818062CFCFCF93DF93C4
:10065000EC01888D8823B9F0AA89BB89E889F989DA
:100660008C9185FD03C0808186FD0DC00FB607FC0F
:10067000F7CF8C9185FFF2CF808185FFEDCFCE0142
:100680000E94B702E9CFDF91CF910895833081F0C6
:1006900028F4813099F08230A9F008958730A9F0CC
:1006A0008830C9F08430B1F4809180008F7D03C020
:1006B000809180008F7780938000089584B58F7734
:1006C00084BD089584B58F7DFBCF8091B0008F7776
:1006D0008093B00008958091B0008F7DF9CFCF93C3
:1006E000DF93ECE7F3E08491E8E6F3E0D491E4E50E
:1006F000F3E0C491CC23A1F081110E944603EC2FBA
:10070000F0E0EE0FFF1FE55CFC4FA591B491EC917A
:10071000ED2381E090E009F480E0DF91CF9108952E
:1007200080E090E0FACF1F93CF93DF93282F30E043
:10073000F901E359FC4F8491F901E75AFC4FD49138
:10074000F901EB5BFC4FC491CC23A9F0162F81116A
:100750000E944603EC2FF0E0EE0FFF1FE556FD4F21
:10076000A591B4918FB7F894EC91111108C0D09570
:10077000DE23DC938FBFDF91CF911F910895DE2B95
:10078000F8CFCF93DF9390E0FC01E75AFC4F249120
:100790008B5B9C4FFC0184918823D1F090E0880F03
:1007A000991FFC01EF56FD4FA591B491FC01E55650
:1007B000FD4FC591D49161110EC09FB7F8948C91F3
:1007C000E22FE0958E238C932881E223E8839FBF5C
:1007D000DF91CF9108958FB7F894EC91E22BEC93D1
:1007E0008FBFF6CF3FB7F894809163029091640277
:1007F000A0916502B091660226B5A89B05C02F3F67
:1008000019F00196A11DB11D3FBFBA2FA92F982F36
:100810008827BC01CD01620F711D811D911D42E031
:10082000660F771F881F991F4A95D1F708958F92F9
:100830009F92AF92BF92CF92DF92EF92FF926B01A5
:100840007C010E94F2034B015C01C114D104E1045C
:10085000F104B9F00E94F203681979098A099B0929
:10086000683E73408105910580F321E0C21AD108EA
:10087000E108F10888EE880E83E0981EA11CB11CE7
:10088000E4CFFF90EF90DF90CF90BF90AF909F901C
:100890008F9008958F929F92AF92BF92EF92FF92A6
:1008A0001F93CF93DF93C82F1092540410925504D6
:1008B00010925604109257041092580461E08FE091
:1008C0000E94C10360E08FE00E9493036C2F70E0F0
:1008D00090E080E00E94170460E08FE00E94C10376
:1008E0008BE990E00197F1F7C0E9D1E00E946F0336
:1008F000892B71F42197D1F78EEF9FEFDF91CF9184
:100900001F91FF90EF90BF90AF909F908F900895B0
:10091000C0E9D1E00E946F03019719F42197D1F744
:10092000EBCFD8E2C0E810E090E9E92EFF24F39481
:100930000E946F03892B29F481E0E81AF108C1F7BE
:10094000DBCF0E94F2034B015C0180E9E82EFF241B
:10095000F3940E946F03019729F481E0E81AF108EB
:10096000C1F7CACF0E94F203681979098A099B0965
:10097000693271058105910538F0E12FF0E0E45B03
:10098000FB4F80858C2B8087C69511F41F5FC0E8D4
:10099000D15051F690E080E0B1CF8F929F92AF920C
:1009A000BF92CF92DF92EF92FF920F931F93CF935C
:1009B000DF938AE0882E912CD0E0C0E0CC24CA944A
:1009C00093E0D92EEE24EA9423E0F22EB12CA12C50
:1009D00010E000E080910D0120E4829FC00111240D
:1009E000816080937C0080917A00806480937A009B
:1009F00080917A0086FDFCCF9091780080917900FB
:100A00008927982789270817190790F1A816B9068A
:100A100008F45C018E159F0568F18C159D0508F49E
:100A20006C01C80FD91F65E070E080E090E00E9483
:100A3000170481E0881A910869F60A0D1B1DCE0182
:100A4000801B910B8C199D098E199F0966E070E03F
:100A50000E94B82CCB01DF91CF911F910F91FF9095
:100A6000EF90DF90CF90BF90AF909F908F900895C0
:100A70008C01D0CF7C01D5CF2FB7F89460915F0265
:100A80007091600280916102909162022FBF08957F
:100A900008958091970290919802891B990B08956F
:100AA000089520913B02260F3327331F2132310551
:100AB000ECF42091BF02FC0190E080E0243069F06A
:100AC00082E00895A0913B022191AC01455E5D4F0B
:100AD000A40FB52FB11D2C930196861798F3809122
:100AE0003B02680F60933B0280E0089581E0089527
:100AF0001092BF0281E08093BE021092990261E0E1
:100B000082E10E94930361E083E10E949303E9EB99
:100B1000F0E080818E7F808380818D7F808388E478
:100B20008093B80085E48093BC00089510929802E9
:100B3000109297021092C6021092E8020E94780565
:100B40008DE192E090937602809375028EE192E0BF
:100B500090937402809373020895CF93DF9391E092
:100B600090931A028823B9F0C091B800D091BA00CE
:100B70008091BC008A7B8093BC0060E082E10E948F
:100B8000930360E083E10E9493030E947805D09371
:100B9000BA00C093B800DF91CF910895CF92DF9251
:100BA000EF92FF920F931F93CF93DF93D091E802C0
:100BB00081E0D13208F09CC0C091E7020E94F203AC
:100BC0006B017C018091BF0281116CC082E0809337
:100BD000BF0281E08093BE028FEF8093BD0210922E
:100BE000BC02D093BB02A7ECB2E0EBE9F2E080E0FC
:100BF000D8138DC010929A0280919A02CC0FC82B04
:100C0000C0939A0280919902813009F084C01092B9
:100C100099020E94F2036B017C0180919A028093F9
:100C2000BB008091C1029091C202A091C302B09119
:100C3000C402892B8A2B8B2BA1F00E94F203009116
:100C4000C1021091C2022091C3023091C4026C19FA
:100C50007D098E099F09061717072807390708F429
:100C600042C08091BC0083FDD8CF85EC8093BC004E
:100C70000E94F2036B017C018091BF02823009F473
:100C80004CC08091BD028F3F09F469C08091BD02C4
:100C9000803209F466C08091BD02803309F463C0DC
:100CA00084E026C08091C1029091C202A091C3024B
:100CB000B091C402892B8A2B8B2B09F483CF0E941D
:100CC000F2030091C1021091C2022091C30230913F
:100CD000C4026C197D098E099F090617170728079A
:100CE000390708F06FCF8091C0020E94AD0585E002
:100CF0001092C6021092E8021092C502DF91CF91C5
:100D00001F910F91FF90EF90DF90CF9008959D91EC
:100D100091938F5F6DCF85EEA9CF8091C1029091A5
:100D2000C202A091C302B091C402892B8A2B8B2BE3
:100D300009F4A2CF0E94F2030091C1021091C202F5
:100D40002091C3023091C4026C197D098E099F095C
:100D5000061717072807390708F08ECFC4CF80E0A1
:100D6000C7CF82E0C5CF83E0C3CFCF92DF92EF92AF
:100D7000FF920F931F93CF93DF93D82FC62F61322B
:100D800008F098C00E94F2036B017C018091BF02C1
:100D900081116BC081E08093BF028093BE029FEF00
:100DA0009093BD021092BC029C0F9093BB02809363
:100DB0009A0280919A02DD0FD82BD0939A028091EB
:100DC0009902813009F078C0109299020E94F203D2
:100DD0006B017C0180919A028093BB008091C102DB
:100DE0009091C202A091C302B091C402892B8A2BB8
:100DF0008B2BA1F00E94F2030091C1021091C2025C
:100E00002091C3023091C4026C197D098E099F099B
:100E1000061717072807390708F448C08091BC0057
:100E200083FDD8CF85EC8093BC000E94F2036B0158
:100E30007C018091BF02813009F440C08091BC02E6
:100E40008C1710F4C091BC02EBE9F2E0A7E7B2E026
:100E500080E08C1355C08C2FDF91CF911F910F91A3
:100E6000FF90EF90DF90CF9008958091C102909114
:100E7000C202A091C302B091C402892B8A2B8B2B92
:100E800009F484CF0E94F2030091C1021091C202C2
:100E90002091C3023091C4026C197D098E099F090B
:100EA000061717072807390708F070CF8091C0028E
:100EB0000E94AD05C0E0CFCF85EEB5CF8091C102D5
:100EC0009091C202A091C302B091C402892B8A2BD7
:100ED0008B2B09F4AECF0E94F2030091C102109156
:100EE000C2022091C3023091C4026C197D098E099F
:100EF0009F09061717072807390708F09ACFD6CF9A
:100F000091919D938F5FA5CF0895E0919802809174
:100F10009702E81730F4F0E0E958FD4F808190E047
:100F200008958FEF9FEF0895CF92DF92EF92FF9297
:100F30000F931F93CF93DF937C01CB018A01209104
:100F4000C502222389F0EB016B01C40ED51ECC151E
:100F5000DD0569F06991D701ED91FC910190F08177
:100F6000E02DC7010995F3CF642F0E945105C801F8
:100F7000DF91CF911F910F91FF90EF90DF90CF9075
:100F80000895CF93DF931F92CDB7DEB76983209189
:100F9000C5022223F9F02091E802203258F021E026
:100FA00030E0FC013383228390E080E00F90DF91FA
:100FB000CF9108958091C602E82FF0E0E953FD4FEC
:100FC000998190838F5F8093C6028093E80281E0CD
:100FD00090E0ECCF61E0CE0101960E945105F7CF81
:100FE000CF93C82F83E50E9413026DE286E893E059
:100FF0000E94C1076C2F86E893E00E94C107CF9141
:101000000C94CE0590E080E00895FC0124813581A8
:10101000232B11F00C944D0208950E94B5061092F6
:101020009802809397020895CF93C82F87E70E9474
:1010300013026C2F86E893E00E94C1070E94CE0540
:1010400087E70E94130261E070E087E790E00E946A
:101050000D080E940002C82F0E94CE058C2FCF9150
:101060000895CF93DF93C82F87E70E9413026C2F58
:1010700086E893E00E94C1070E94CE0587E70E94A0
:10108000130262E070E087E790E00E940D080E9482
:101090000002D82F80E0C82F0E940002C82BD92B55
:1010A0000E94CE05CE01DF91CF91089587E70E947F
:1010B000130264EF86E893E00E94C1076EE286E8BF
:1010C00093E00E94C1070E94CE0565E070E080E0D9
:1010D00090E00E94170486EF0C9431084F925F92C3
:1010E0006F927F928F929F92AF92BF92CF92DF9238
:1010F000EF92FF92CF93DF9300D000D01F92CDB735
:10110000DEB70E9456084C01B12CA12C209121047D
:101110002295220F220F207C2C5C298387E70E94D6
:10112000130264EF86E893E00E94C107698186E8B4
:1011300093E00E94C1070E94CE0580912104811195
:1011400074C165E070E080E090E00E94170486EFD3
:101150000E943108B0E0A0E0CC24D82EE92EFA2E6F
:1011600088EF0E941408A7019601282B29833A834F
:101170004B835C83309121043D83809136049091B0
:101180003704A5019401281B390B41095109A0918D
:101190003404B09135040E94C6284B015C01AFE0D5
:1011A000B594A79497948794AA95D1F760912E044B
:1011B00070912F04072E000C880B990BBBE0660F73
:1011C000771F881F991FBA95D1F72091300430916D
:1011D0003104032E000C440B550B280D391D4A1DFC
:1011E0005B1D0E94A728820E931EA41EB51E7501CA
:1011F000640140EAC41A4FE0D40AE108F108A701EB
:101200009601C701B6010E94A82C4B015C018CE03D
:10121000B594A794979487948A95D1F7A0912604C2
:10122000B09127040E94D1282B013C019DE07594C8
:101230006794579447949A95D1F7A0912804B09158
:101240002904A50194010E94D1289C01552737FD4E
:101250005095452F240D351D461D571D2E5F3F4FC0
:101260004F4F5F4F62E055954795379527956A95A3
:10127000D1F730584F4F5F4FA0913204B0913304F3
:101280000E94C6282B013C017FE076946794579416
:1012900047947A95D1F788E090E05D81851B9109AC
:1012A00029813A814B815C8104C0569547953795D9
:1012B00027958A95D2F729833A834B835C83A09143
:1012C0002A04B0912B04A50194010E94D1284B015E
:1012D0005C01EBE0B594A79497948794EA95D1F7D5
:1012E000A0912404B0912504A70196010E94D12861
:1012F000FBE09595879577956795FA95D1F7680DF9
:10130000791D8A1D9B1D8090220490902304092C36
:10131000000CAA08BB08A2E0880C991CAA1CBB1CE4
:10132000AA95D1F7680D791D8A1D9B1D0D8004C0FB
:10133000660F771F881F991F0A94D2F76E5F7F4F41
:101340008F4F9F4F24E030E040E050E00E94A728FC
:1013500089819A81AB81BC81821B930BA40BB50B55
:101360009C01AD0160E573EC80E090E00D8004C06D
:1013700096958795779567950A94D2F70E94A82C41
:1013800097FD66C0660F771F881F991FA301920102
:101390000E94102969017A019927F7FC9A958F2DEF
:1013A0007E2D6D2D9B01AC010E94A82C9B01AC01F0
:1013B000AEEDBBE00E94C6284B015C01A3E4B3EE96
:1013C000A70196010E94D428BC01992777FD90952A
:1013D000892F4501BB2497FCB094AB2C680D791D77
:1013E0008A1D9B1D6153714F8F4F9F4F44E0959510
:1013F0008795779567954A95D1F76C0D7D1D8E1D64
:101400009F1D0F900F900F900F900F90DF91CF9135
:10141000FF90EF90DF90CF90BF90AF909F908F9014
:101420007F906F905F904F900895813029F468E02D
:1014300070E080E090E089CE823029F46EE070E0C8
:1014400080E090E082CE6AE170E080E090E07DCEC6
:10145000A30192010E94102969017A01CC0CDD1CC4
:10146000EE1CFF1C99CFAF92BF92DF92EF92FF92DA
:101470000F931F93CF93DF935C0102E913E0D0E059
:10148000C0E0F801D1908F017501EC0EFD1EC7017F
:101490000E949128D81621F06D2DC7010E9499282D
:1014A0002196CC34D10569F782E993E0DF91CF91A1
:1014B0001F910F91FF90EF90DF90BF90AF90089534
:1014C000FC0180819181009711F00C94102360E061
:1014D00070E0CB010895FB0144815581FC0124811A
:1014E00035812417350778F080819181009759F074
:1014F000FB01608171816115710529F00E94CC2E7C
:1015000021E0892B09F020E0822F08950F931F938B
:10151000CF93DF938C01EB01FC01808191810097D7
:10152000E1F06881798161157105A9F042815381EB
:101530002C813D814217530770F00E94C52E8C818B
:101540009D81F801958384831D821C82DF91CF9158
:101550001F910F9108950E946E2D88819981F80145
:10156000918380838A819B81938382838C819D81F7
:1015700095838483198218821B821A82E5CFCF93C8
:10158000DF93EC0188819981009711F00E946E2D04
:10159000198218821D821C821B821A82DF91CF91D0
:1015A0000895FC0180819181009711F00C946E2DBB
:1015B00008950C946E2D0F931F93CF93DF93EC013E
:1015C00088819981009759F02A813B812617370736
:1015D00030F081E0DF91CF911F910F9108958B0141
:1015E0006F5F7F4F0E94F72D009759F09983888392
:1015F0001B830A832C813D81232B59F7FC01108228
:10160000E8CF80E0E7CFEF92FF920F931F93CF9345
:10161000DF936115710541F480E0DF91CF911F9157
:101620000F91FF90EF90089541155105B1F07B01A6
:10163000EC010C811D81040F151FB8010E94DB0A0B
:10164000882351F3288139818C819D81B701820FD4
:10165000931F0E94C52E1D830C8381E0DECFCF93A4
:10166000DF93EC01FB0101900020E9F73197AF0116
:10167000461B570B0E94030B811103C0CE010E9431
:10168000BF0ACE01DF91CF910895CF93DF93EC0194
:10169000FB0144815581608171810E94030B81119E
:1016A00003C0CE010E94BF0ACE01DF91CF91089501
:1016B000FB0101900020E9F73197AF01461B570B62
:1016C0000C94030BFB0144815581608171810C9462
:1016D000030BEF92FF920F931F93CF93DF93EC01D5
:1016E0008B01CB010E943E237C01BC01CE010E94F4
:1016F000DB0A81110BC0CE010E94BF0ACE01DF912F
:10170000CF911F910F91FF90EF900895FD82EC8291
:10171000B801888199810E943723F0CFFC011182A2
:10172000108213821282158214820C94690BEF923C
:10173000FF920F931F93CF93DF93EC017B018A01FC
:10174000BA010E94DB0A81110BC0CE010E94BF0AC0
:10175000CE01DF91CF911F910F91FF90EF900895EF
:101760001D830C83B701888199810E94C52EF0CF1B
:10177000FB0101900020E9F73197AF01461B570BA1
:101780000C94970B0F931F93CF93DF93CDB7DEB7D6
:1017900062970FB6F894DEBF0FBECDBF8C01CB01B0
:1017A000F8011182108213821282158214824AE09B
:1017B000BE016F5F7F4F0E944723BE016F5F7F4F67
:1017C000C8010E94B80B62960FB6F894DEBF0FBE38
:1017D000CDBFDF91CF911F910F910895CF93DF93EC
:1017E000EC01FB018617970749F060817181611553
:1017F000710541F0448155810E94970BCE01DF9124
:10180000CF9108950E94BF0AF9CFFC011182108286
:1018100013821282158214820C94EE0BFC01118249
:1018200010821382128215821482FB010190002023
:10183000E9F73197AF01461B570B0C94970BCF92EA
:10184000DF92EF92FF920F931F93CF93DF936C0180
:101850007B018A014617570720F48F2D7A01062F46
:10186000182F68E471E0C6010E940E0CC091FA03C3
:10187000D091FB03EC16FD06F8F40C171D0708F4D5
:10188000E801E091F603F091F703EC0FFD1F1081E2
:1018900010826091F6037091F7036E0D7F1DC601F3
:1018A0006115710599F00E94B80B8091F603909133
:1018B000F703C80FD91F1883C601DF91CF911F917D
:1018C0000F91FF90EF90DF90CF9008950E94BF0A94
:1018D000ECCFEF92FF920F931F93CF93DF93CDB78F
:1018E000DEB7A1970FB6F894DEBF0FBECDBF7C0167
:1018F000CB01BA01F7011182108213821282158284
:10190000148242E0420F8E010F5F1F4F0E94EE22B1
:10191000009789F0BC01C7010E94B80BA1960FB6D1
:10192000F894DEBF0FBECDBFDF91CF911F910F9115
:10193000FF90EF900895C7010E94BF0AEFCF8F92EA
:101940009F92AF92BF92EF92FF920F931F93CF930C
:10195000DF93CDB7DEB72C970FB6F894DEBF0FBE7E
:10196000CDBF64E670E080E090E00E9417048091B3
:101970000301909104010B9731F58091590488235C
:1019800009F0F89482E10E944A048C018091590484
:10199000882309F078940115110509F4BDC080E091
:1019A00090ECA9E7B4EC80934C0490934D04A09381
:1019B0004E04B0934F048093500490935104A0932D
:1019C0005204B0935304809103019091040146970F
:1019D00031F580915904882309F0F89481E00E9440
:1019E0004A048C0180915904882309F078940115E8
:1019F000110509F4F2C080E090ECA9E7B4EC809303
:101A00004C0490934D04A0934E04B0934F048093E4
:101A1000500490935104A0935204B093530464E68D
:101A200070E080E090E00E941704012B09F063C091
:101A300040915004509151046091520470915304AC
:101A400021E0CE0107960E94690C69E471E0CE01A5
:101A500001960E940E0CBE01695F7F4FCE01019678
:101A60000E94450B6CE471E00E942F0BBC0182E0E8
:101A700094E00E94EE0BCE0101960E94D10A4091A3
:101A80004C0450914D0460914E0470914F0421E03C
:101A9000CE0101960E94690CBE016F5F7F4FCE019F
:101AA00007960E94860ACE0101960E94D10A60E53F
:101AB00071E0CE0101960E940E0CBE01695F7F4F5E
:101AC000CE0101960E94450B63E571E00E942F0B49
:101AD000BC0182E094E00E94620BCE0101960E945C
:101AE000D10A64E670E080E090E00E941704CE0125
:101AF00007960E94D10A2C960FB6F894DEBF0FBE4F
:101B0000CDBFDF91CF911F910F91FF90EF90BF90CC
:101B1000AF909F908F90089510915404E0905504D9
:101B20006E2D70E090E080E00E9471272DEC3CEC7F
:101B30004CEC5DE30E94D0274B015C01612F70E00B
:101B400090E080E00E9471279B01AC01C501B401C7
:101B50000E94422960934C0470934D0480934E047C
:101B600090934F0400915604F0905704602F6F77C4
:101B700070E090E080E00E9471274B015C016F2DC6
:101B800070E090E080E00E9471272DEC3CEC4CEC82
:101B90005DE30E94D0279B01AC01C501B4010E9406
:101BA000422907FD18C0609350047093510480933C
:101BB0005204909353041E0D100F1F0D81E090E00E
:101BC00020915804121302C090E080E000271127F2
:101BD000081B190BF8CE9058E6CF109155040091D0
:101BE0005404609154047091550476276727762732
:101BF00090E080E00E946F272DEC3CEC4CEC5DE324
:101C00000E94D02760934C0470934D0480934E043F
:101C100090934F04E0905704F09056046F2D6F7727
:101C2000762F6E2D90E080E00E946F272DEC3CEC2B
:101C30004CEC5DE30E94D027F7FC18C06093500481
:101C4000709351048093520490935304100F1E0D0F
:101C50001F0D81E090E020915804121302C090E023
:101C600080E000271127081B190BD9CE9058E6CF2A
:101C70000F931F93CF93DF938C01EB0188E2FB015D
:101C800011928A95E9F74BE050E065E571E0CE01ED
:101C90000E94DA2E1B8681E090E0A0E0B0E08C8705
:101CA0009D87AE87BF87F80185899689A789B08D02
:101CB000888B998BAA8BBB8B82E090E0A0E0B0E090
:101CC0008C8B9D8BAE8BBF8B1CA21DA21EA21FA254
:101CD00080E090E0A8E4B4E4888F998FAA8FBB8F4E
:101CE00080E090E0A8E4B4EC8C8F9D8FAE8FBF8F26
:101CF0008DEC9CECACE4BEE388A399A3AAA3BBA3A0
:101D0000DF91CF911F910F910895AF92BF92CF9223
:101D1000DF92EF92FF920F931F93CF93DF938C018B
:101D2000EB0184E2FB0111928A95E9F78EE10E94B2
:101D3000130263E086E893E00E94C1070E94CE058B
:101D400066E08EE10E94B506109298028093970299
:101D50008630F0F30E940002A82E0E940002B82EE6
:101D60000E940002E82E0E940002F82E0E9400024B
:101D7000C82E0E940002D82E60E07A2D6B29072E13
:101D8000000C880B990B0E947127F80165837683FC
:101D90008783908760E07C2D6D29072E000C880BCF
:101DA000990B0E947127F801618772878387948756
:101DB00060E07E2D6F29072E000C880B990B0E9486
:101DC0007127F801658776878787908B118A128A39
:101DD000138A148A84E290E0A0E0B0E088839983BB
:101DE000AA83BB8385899689A789B08D8C839D83BF
:101DF000AE83BF8382E090E0A0E0B0E0888799875F
:101E0000AA87BB87188A198A1A8A1B8A20E030E8B9
:101E100049E854E465817681878190850E94202A73
:101E200020E030E048EC52E40E94D0276C8B7D8BA0
:101E30008E8B9F8B20E030E849E854E4F8016185FF
:101E40007285838594850E94202A20E030E048EC4A
:101E500052E40E94D027688F798F8A8F9B8F20E071
:101E600030E045E754E4F8016585768587859089FB
:101E70000E94202A20E030E048EC52E40E94D02763
:101E80006C8F7D8F8E8F9F8F81E0DF91CF911F911F
:101E90000F91FF90EF90DF90CF90BF90AF9008959B
:101EA00085ED8093BC008091C1029091C202A09107
:101EB000C302B091C4020796A11DB11D23E0B695DF
:101EC000A795979587952A95D1F72091BC0024FD79
:101ED00003C01092BF0208954091C1025091C20206
:101EE0006091C3027091C402452B462B472B69F3C6
:101EF0000097A105B10541F025E32A95F1F700000F
:101F00000197A109B109E1CF8091C0020C94AD0500
:101F10004F925F926F927F928F929F92AF92BF92F9
:101F2000CF92DF92EF92FF920F931F93CF93DF93A5
:101F3000CDB7DEB7C654D1090FB6F894DEBF0FBED9
:101F4000CDBF8C0168E471E0CE01C7960E940E0CF3
:101F500068E471E0CE01CD960E940E0CBE016F5F69
:101F60007F4F88E094E00E94850E20E030E040E260
:101F700051E46D897E898F89988D0E94D0272B012D
:101F80003C0120E030E040E251E4698D7A8D8B8D98
:101F90009C8D0E94D0274B015C0120E030E040E2A4
:101FA00051E46D8D7E8D8F8D98A10E94D02727964C
:101FB0006CAF7DAF8EAF9FAF2797C301B201905832
:101FC000A50194010E94C1292BED3FE049EC5FE39C
:101FD0000E9442292091A2033091A3034091A403BF
:101FE0005091A5030E9442296B017C0120E030E062
:101FF000A9010E946A2787FF0AC02BED3FE049EC48
:1020000050E4C701B6010E9442296B017C012BED0F
:102010003FE049EC50E4C701B6010E94EF2A1816D0
:1020200054F42BED3FE049EC50E4C701B6010E94A7
:1020300041296B017C0120E030E044E353E4C70117
:10204000B6010E94D0272BED3FE049E450E40E9406
:10205000202A6B017C010E94922ACE018B960E945D
:10206000C20B6DE571E0CE0185960E940E0CBE019B
:10207000655D7F4FCE0185960E94450B67E671E056
:102080000E942F0BBC0182E094E00E94EE0BCE0177
:1020900085960E94D10ACE018B960E94D10A20E03B
:1020A00030E044EB52E4C701B6010E946A271816DB
:1020B0000CF4A0C120E030E040E05FE3C701B601CE
:1020C0000E9442290E94922ACE018B960E94C20B46
:1020D0006EE671E0CE0185960E940E0CBE01655D34
:1020E0007F4FCE0185960E94450BBC01CE01C7965D
:1020F0000E94EE0BCE0185960E94D10ACE018B96EE
:102100000E94D10A61E771E0CE01CD960E94B80B22
:102110006CE671E0CE0185960E940E0CBE01635CF8
:102120007F4FCE0185960E94450BBC01CE01C7961C
:102130000E94620BCE0185960E94D10A0E943C0546
:10214000C0901602D0901702E0901802F090190289
:102150006C197D098E099F090E946F2720E030E0ED
:102160004AE754E40E94202AAB01BC0123E0CE01DF
:102170008B960E94690C64E871E0CE0185960E94FE
:102180000E0CBE01655D7F4FCE0185960E94450B0A
:1021900068E771E00E942F0BBC018AEE93E00E9479
:1021A000EE0BCE0185960E94D10ACE018B960E943D
:1021B000D10A6AEE73E0CE0185960E94050C62E0BA
:1021C00074E0CE0185960E94450BBE01695C7F4F8D
:1021D0000E94450BBC01CE01C7960E94EE0BCE01BA
:1021E00085960E94D10A66E872E082E094E00E943F
:1021F000690B21E0B301A201CE0185960E94690C12
:10220000BE016B5D7F4F82E094E00E94620BCE01C5
:1022100085960E94D10A21E027964CAD5DAD6EAD4A
:102220007FAD2797CE01C1960E94690C21E0B501D0
:10223000A401CE018B960E94690C6CE671E0CE0180
:1022400085960E940E0CBE01655D7F4FCE0185967E
:102250000E94450B6CE671E00E942F0BBE016F5C83
:102260007F4F0E94450B6BE771E00E942F0BBC0172
:1022700082E094E00E94620BCE0185960E94D10A12
:10228000CE018B960E94D10ACE01C1960E94D10A3E
:10229000A3019201C301B2010E94D0276B017C010E
:1022A000A5019401C501B4010E94D0279B01AC0196
:1022B000C701B6010E9442296B017C0127962CAD13
:1022C0003DAD4EAD5FAD2797CA01B9010E94D02741
:1022D0009B01AC01C701B6010E9442290E94522B0A
:1022E0006B017C016FE771E082E094E00E94580B83
:1022F00021E0B701A601CE0185960E94690CBE01BE
:102300006B5D7F4FCE018B960E94050C6CE771E0F0
:10231000CE018B960E942F0BBC0182E094E00E94BC
:10232000620BCE018B960E94D10ACE0185960E9447
:10233000D10A20E030E64AE656E4C701B6010E9421
:102340006A27BE01695C7F4F87FFC1C0CE018596B9
:102350000E94050C63E871E0CE0185960E942F0B68
:1023600062E074E00E94450BBC0182E094E00E94B0
:10237000EE0BCE0185960E94D10A03301105A1F41F
:1023800062E074E0CE0185960E94050CCE01859630
:102390000E940508CE0185960E94D10A68E471E08A
:1023A00082E094E00E94B80B6AE070E080E090E088
:1023B0000E941704CE01CD960E94D10ACE01C79685
:1023C0000E94D10ACA5BDF4F0FB6F894DEBF0FBE82
:1023D000CDBFDF91CF911F910F91FF90EF90DF90D4
:1023E000CF90BF90AF909F908F907F906F905F90B5
:1023F0004F90089520E030E044E353E4C701B60174
:102400000E946A2718168CF0A701960160E070E818
:1024100084E393E40E9441290E94922ACE018B9684
:102420000E94C20B63E771E055CE20E030E047E840
:1024300053E4C701B6010E946A2718168CF120E008
:1024400030E044E353E4C701B6010E94412920E093
:1024500030E040E05FE30E9442290E94922ACE01D0
:102460008B960E94C20B63E771E0CE0185960E94B5
:102470000E0CBE01655D7F4FCE0185960E94450B17
:10248000BC01CE01C7960E94EE0BCE0185960E943C
:10249000D10ACE018B960E94D10A66E771E034CE54
:1024A000A701960160E070E084EB93E40E9441296B
:1024B00020E030E040E05FE30E9442290E94922A3F
:1024C000CE018B960E94C20B6EE671E0CECF82E009
:1024D00094E00E94EE0B68CF4F925F926F927F92D2
:1024E0008F929F92AF92BF92CF92DF92EF92FF9224
:1024F000CF93DF93CDB7DEB72C970FB6F894DEBF3E
:102500000FBECDBF0E946E086B017C010E94560871
:102510009C0150E040E0E1E2F4E085899689281BC7
:10252000390B41095109A389B4890E94C6284B017E
:102530005C018FE0B594A794979487948A95D1F71E
:1025400065857685072E000C880B990B2BE0660FAE
:10255000771F881F991F2A95D1F727853089032E69
:10256000000C440B550B280D391D4A1D5B1D0E94A4
:10257000A728CA01B901680D791D8A1D9B1D685FD6
:102580007F4F8F4F9F4F34E095958795779567954F
:102590003A95D1F70E9471272B013C0160919E036F
:1025A00070919F038091A0039091A1030E947127D5
:1025B0004B015C010E946E080E947127A5019401E5
:1025C0000E94202A21E03EED42E45EE30E94FC2AC4
:1025D0004B015C01C701B6010E94712720E030E089
:1025E00048EC52E40E94202AAB01BC0122E0CE015B
:1025F00001960E94690CBE016F5F7F4F8AEE93E0E7
:102600000E94860ACE0101960E94D10A6EE072E015
:102610008AEE93E00E94580B6AEE73E080EF93E03D
:102620000E94EE0B6DEE71E0CE0101960E940E0C41
:102630006AEE73E0CE0101960E94450BBC018AEE62
:1026400093E00E94EE0BCE0101960E94D10A6AE54A
:1026500072E082E094E00E94690B20E030E040E20A
:1026600051E4C301B2010E94202AAB01BC0121E068
:10267000CE0101960E94690CBE016F5F7F4F82E020
:1026800094E00E94620BCE0101960E94D10A66E896
:1026900071E082E094E00E94580BA501940160E093
:1026A00070E080E89FE30E94412920E03AE24DE299
:1026B00057E40E94D027AB01BC0121E0CE01019676
:1026C0000E94690CBE016F5F7F4FCE0107960E948A
:1026D000050C6CE871E0CE0107960E942F0BBC013F
:1026E00082E094E00E94620BCE0107960E94D10A1C
:1026F000CE0101960E94D10A6AEE73E0CE010196E6
:102700000E94050C6CE671E0CE0101960E942F0B31
:1027100062E074E00E94450BBC0182E094E00E94FC
:10272000EE0BCE0101960E94D10A65E070E080E0D8
:1027300090E00E9417042C960FB6F894DEBF0FBEEF
:10274000CDBFDF91CF91FF90EF90DF90CF90BF9002
:10275000AF909F908F907F906F905F904F90089573
:102760002F923F924F925F926F927F928F929F92A1
:10277000AF92BF92CF92DF92EF92FF920F931F938F
:10278000CF93DF93CDB7DEB7C056D1090FB6F8941B
:10279000DEBF0FBECDBF2D966CAF7DAF8EAF9FAFAE
:1027A0002D9761962CAF3DAF4EAF5FAF6197683EFE
:1027B0007340810591055CF018E2E12EF12C00E0F8
:1027C00010E02D96ECAEFDAE0EAF1FAF2D976196CB
:1027D000ECACFDAC0EAD1FAD6197E11421EEF2063D
:1027E000054F15405CF0E12C11EEF12E05EF15E0E0
:1027F0006196ECAEFDAE0EAF1FAF61978091720295
:10280000882351F0E12CF12C8701E3946196ECAE22
:10281000FDAE0EAF1FAF61970E943C056D966CAF89
:102820007DAF8EAF9FAF6D970E943C0569966CAFF0
:102830007DAF8EAF9FAF69976D966CAD7DAD8EAD60
:102840009FAD6D9728EE33E040E050E00E94A7284E
:10285000A1962CAF3DAF4EAF5FAFA19701E026969A
:102860000FAF269765961CAE1DAE1EAE1FAE6597C8
:102870001E0117E0210E311C69966CAD7DAD8EAD49
:102880009FAD69976D96ECACFDAC0EAD1FAD6D972D
:102890006E197F09800B910B6196ECACFDAC0EAD0F
:1028A0001FAD61976E157F05800791070CF060C31F
:1028B0000E94712720E030E04AE754E40E94202A79
:1028C000AB01BC0123E0CE0101960E94690CBE0160
:1028D0006F5F7F4F80EF93E00E94860ACE010196E2
:1028E0000E94D10A61960CAD1DAD2EAD3FAD619732
:1028F0000A3011052105310524F518AA1FA61AAAC8
:1029000019AA1CAA1BAA2AE0AE014F5F5F4FA1962D
:102910006CAD7DAD8EAD9FADA1970E945223BE01DF
:102920006F5F7F4FCE018F960E94B80BBE01615D35
:102930007F4F80EF93E00E94860ACE018F960E941F
:10294000D10A80917202882361F168E471E080EF1E
:1029500093E00E94B80B83E50E94130262E386E8CD
:1029600093E00E94C1070E94CE0583E50E941302F6
:1029700066E070E083E590E00E940D0808E314E053
:10298000C801885394400F5F1F4F309197022091E8
:102990009802321701F10E940002D8011D968C9313
:1029A000EFCF64E871E0CE0101960E940E0C60EF5B
:1029B00073E0CE0101960E94450B68E771E00E942A
:1029C0002F0BBC0180EF93E00E94EE0BCE0101962D
:1029D0000E94D10AC0CF069729F010923804B1E0C6
:1029E000B09339040E94CE0580914604909147042B
:1029F0009A83898380914804909149049C838B83B6
:102A000080914A0490914B049E838D83FE01319600
:102A10005F019AE3892E94E0992E3E01F3E26F0E56
:102A2000711C8301D5016D917D915D01F401C1900F
:102A3000D190E190F1904F01072E000C880B990B7B
:102A40000E947127A70196010E94D027D8016D939B
:102A50007D938D939D938D01A214B30419F76DE4BA
:102A600072E082E094E00E94690B8301045F1F4FD3
:102A7000C12CD12C7601F30181909190A190B1905D
:102A80003F01A5019401C501B4010E94D0279B011B
:102A9000AC01C701B6010E9442296B017C0123E011
:102AA000B501A401CE0101960E94690CBE016F5FC1
:102AB0007F4FCE018F960E94050C6CE671E0CE012F
:102AC0008F960E942F0BBC0182E094E00E94620B63
:102AD000CE018F960E94D10ACE0101960E94D10AA2
:102AE0006016710641F6C701B6010E94522B2B01F8
:102AF0003C0123E0BC01A201CE018F960E94690C2B
:102B000067E471E0CE0101960E940E0C60EF73E065
:102B1000CE0101960E94450B6EE871E00E942F0BDA
:102B2000BE01615D7F4F0E94450B61E971E00E942B
:102B30002F0BBC0182E094E00E94620BCE01019653
:102B40000E94D10ACE018F960E94D10ACBA4DCA4A8
:102B5000EDA4FEA48BA09CA0ADA0BEA00FA118A5C3
:102B600029A53AA525960CAF1DAF2EAF3FAF2597EF
:102B70002DEC3CEC4CE45FE3C301B2010E94EF2A70
:102B800018160CF07CC12AE939E949E95FE3C30171
:102B9000B2010E946A2787FF72C126961FAD269751
:102BA000112309F46CC120E030E0A901C701B6018E
:102BB0000E946A27882309F44FC1A5019401C50129
:102BC000B4010E94D0272B013C0125962CAD3DADD0
:102BD0004EAD5FAD2597CA01B9010E94D0279B0178
:102BE000AC01C301B2010E9442290E94522BA701ED
:102BF00096010E94C12920EE3EE245E652E40E9481
:102C0000D02729966CAF7DAF8EAF9FAF299720E07C
:102C100030E0A90125966CAD7DAD8EAD9FAD2597B9
:102C20000E946A27882309F41CC1A5019401C501EB
:102C3000B4010E94D0272B013C01A7019601C701D6
:102C4000B6010E94D0279B01AC01C301B2010E94D2
:102C500042290E94522B25962CAD3DAD4EAD5FAD65
:102C600025970E94C12920EE3EE245E652E40E94EB
:102C7000D0272B013C0120E030E0A901C501B401BF
:102C80000E946A27882309F4F1C0A7019601C701B1
:102C9000B6010E94D0276B017C0125962CAD3DAD7D
:102CA0004EAD5FAD2597CA01B9010E94D0279B01A7
:102CB000AC01C701B6010E9442290E94522BA50116
:102CC00094010E94C1296B017C0160EF73E0CE0189
:102CD00001960E94050C64E971E0CE0101960E9404
:102CE0002F0BBC0182E094E00E94EE0BCE01019616
:102CF0000E94D10A21E029964CAD5DAD6EAD7FAD4D
:102D00002997CE01CB960E94690C21E0B301A20164
:102D1000CE01C5960E94690C20EE3EE245E652E4E3
:102D2000C701B6010E94D027AB01BC0121E0CE0152
:102D300001960E94690CBE016F5F7F4FCE018F9696
:102D40000E94050C6CE671E0CE018F960E942F0B5D
:102D5000BE016B5C7F4F0E94450B6CE671E00E94E8
:102D60002F0BBE01655C7F4F0E94450BBC018AEEB4
:102D700093E00E94EE0BCE018F960E94D10ACE0105
:102D800001960E94D10ACE01C5960E94D10ACE01B9
:102D9000CB960E94D10A6AEE73E082E094E00E9432
:102DA000620B2D962CAD3DAD4EAD5FAD2D972B300A
:102DB00031054105510544F46596ECACFDAC0EAD12
:102DC0001FAD659717FDCFC062E074E0CE0101969C
:102DD0000E94050CCE0101960E940508CE010196C5
:102DE0000E94D10A01E026960FAF269768E471E0B1
:102DF00082E094E00E94B80B0E943C057B018C01AC
:102E000069962CAD3DAD4EAD5FAD6997E21AF30A00
:102E1000040B150B6596ECAEFDAE0EAF1FAF6597BC
:102E20002D968CAD9DADAEADBFAD2D97E816F906D4
:102E30000A071B0744F4BC01CD016E197F09800B02
:102E4000910B0E9417040E943C0569966CAF7DAF00
:102E50008EAF9FAF699710CD6BED7FE089EC9FE35C
:102E6000CACE6BED7FE089EC9FE3FDCE8BEDC82EE3
:102E70008FE0D82E89ECE82E8FE3F82E26CF23E0C2
:102E8000B501A401CE018F960E94690C60EF73E03A
:102E9000CE0101960E94050C6CEA71E0CE0101960C
:102EA0000E942F0BBE01615D7F4F0E94450B62E9BE
:102EB00071E00E942F0BBC0180EF93E00E94EE0BAB
:102EC000CE0101960E94D10ACE018F960E94D10AAE
:102ED00023E0B701A601CE01C5960E94690C23E04C
:102EE00025964CAD5DAD6EAD7FAD2597CE010196BB
:102EF0000E94690CBE016F5F7F4FCE018F960E94CA
:102F0000050C6FEA71E0CE018F960E942F0BBE0177
:102F10006B5C7F4F0E94450B62E971E00E942F0BB2
:102F2000BC018AEE93E00E94EE0BCE018F960E94C8
:102F3000D10ACE0101960E94D10ACE01C5960E9407
:102F4000D10A62E074E0CE0101960E94050CCE0128
:102F500001960E940508CE0101960E94D10A26968C
:102F60001FAE269743CF11E026961FAF26973ECF80
:102F7000C05ADF4F0FB6F894DEBF0FBECDBFDF9152
:102F8000CF911F910F91FF90EF90DF90CF90BF9066
:102F9000AF909F908F907F906F905F904F903F90F9
:102FA0002F9008954F925F926F927F928F929F928F
:102FB000AF92BF92CF92DF92EF92FF920F931F9347
:102FC000CF93DF9300D000D000D0CDB7DEB78C0117
:102FD00068E471E082E094E00E94B80BC8010596B5
:102FE000059740F00C3E2FEF120724F010936A0271
:102FF0000093690210161106CCF10F3F3FEF130743
:103000000CF06CC00B3F4FEF1407D4F4093F5FEF97
:1030100015070CF063C0083F8FEF18070CF0C9C00C
:10302000013FEFEF1E070CF059C0083E1F4F09F497
:103030009EC168E772E082E094E00E94690B4EC096
:103040000C3F2FEF120709F4C6C00CF4B5C00D3FBA
:103050001F4F79F781E0809372028091690290910D
:103060006A0290936D0280936C0238C0053011059E
:1030700009F4BCC064F50230110509F4AFC00CF4CA
:1030800095C00330110551F10430110591F681E02E
:1030900080930D010E94CD048C016DE572E082E009
:1030A00094E00E94690B60E074E0601B710BCE013C
:1030B00001960E94C20BBE016F5F7F4F82E094E0D9
:1030C0000E94620BCE0101960E94D10A07C009300E
:1030D0001105ACF5073011050CF492C0809106047F
:1030E00090910704892B71F062E074E0CE010196A3
:1030F0000E94050CCE0101960E940508CE010196A2
:103100000E94D10A64E670E080E090E00E9417041B
:1031100026960FB6F894DEBF0FBECDBFDF91CF91DC
:103120001F910F91FF90EF90DF90CF90BF90AF90E5
:103130009F908F907F906F905F904F90089509308F
:10314000110509F4DBC00138110509F072CF809137
:103150000001882329F10E946C1262E074E0CE0124
:1031600001960E94050CCE0101960E940508CE0131
:1031700001960E94D10A64EF71E080E090E00E9425
:10318000170480917202882309F4F5C021E030E031
:1031900040E050E06AE070E080E090E00E94B01310
:1031A00064EF71E080E090E00E9417040E949F0CA1
:1031B00095CF0E943C0592CF80917202882321F026
:1031C00082E094E00E944D0268EC70E080E090E0C4
:1031D0000E94170483CF1092720280CF8091000169
:1031E000882309F47BCF0E946C1278CF6DE672E0E1
:1031F00082E094E00E94690B0E94CD04BC0157CF8D
:1032000080910001882309F469CF8091720288239C
:1032100029F082E090E00E94880F60CF20E030E04B
:103220004AE754E46091050170910601809107011D
:10323000909108010E94D0270E94922A4B015C01C4
:1032400020E030E04AE754E46091090170910A01FE
:1032500080910B0190910C010E94D0270E94922A2C
:103260006B017C0159EEC51653E0D506E104F1046B
:103270002CF084E1C82ED12CE12CF12C0E943C05CD
:1032800060931602709317028093180290931902AC
:103290000E943C052B013C0180911602909117027F
:1032A000A0911802B0911902A3019201281B390BB9
:1032B0004A0B5B0BDA01C90188159905AA05BB0504
:1032C0000CF00CCF83E090E00E94880F0E943C0538
:1032D000DC01CB0184199509A609B7098C159D0558
:1032E000AE05BF05ACF6A7019601281B390B4A0BAA
:1032F0005B0BCA01B9010E941704CACF809100017B
:10330000882309F4EBCE80917202882359F021E0E2
:1033100030E040E050E06AE070E080E090E00E9441
:10332000B013DCCE20E030E04AE754E460910501C0
:103330007091060180910701909108010E94D027A9
:103340000E94922A6B017C0120E030E04AE754E4BD
:103350006091090170910A0180910B0190910C011B
:103360000E94D0270E94922AA7019601D8CFF0E0B0
:10337000E0E00995B3CE20E030E04AE754E4609104
:1033800005017091060180910701909108010E944A
:10339000D0270E94922A6B017C0120E030E04AE7AE
:1033A00054E46091090170910A0180910B019091A0
:1033B0000C010E94D0270E94922AA7019601EECE0E
:1033C0001F920F920FB60F9211242F933F934F939A
:1033D0005F936F937F938F939F93AF93BF93EF937D
:1033E000FF9389EE92E00E94B702FF91EF91BF91A7
:1033F000AF919F918F917F916F915F914F913F918D
:103400002F910F900FBE0F901F9018951F920F9243
:103410000FB60F9211242F938F939F93EF93FF93E7
:10342000E091F902F091FA028081E091FF02F091BF
:10343000000382FD1BC09081809102038F5F8F7318
:1034400020910303821741F0E0910203F0E0E7517D
:10345000FD4F958F80930203FF91EF919F918F9184
:103460002F910F900FBE0F901F9018958081F4CF71
:103470001F920F920FB60F9211242F933F938F93A9
:103480009F93AF93BF9380915F0290916002A09150
:103490006102B091620230915E0223E0230F2D376A
:1034A00058F50196A11DB11D20935E0280935F0225
:1034B00090936002A0936102B093620280916302D4
:1034C00090916402A0916502B09166020196A11DDF
:1034D000B11D8093630290936402A0936502B09340
:1034E0006602BF91AF919F918F913F912F910F9065
:1034F0000FBE0F901F90189526E8230F0296A11D6E
:10350000B11DD2CF1F920F920FB60F9211242F939D
:103510003F934F935F936F937F938F939F93AF935B
:10352000BF93EF93FF938091B900887F803609F4B1
:103530004AC0F0F5883209F4A7C018F5803109F4C3
:103540009BC0B8F4882309F4F9C0883009F494C00A
:10355000FF91EF91BF91AF919F918F917F916F916B
:103560005F914F913F912F910F900FBE0F901F9041
:103570001895883109F488C0803251F78093BD02D4
:1035800014C0803409F49DC040F48033B9F388330B
:10359000F9F68093BD0285ECB0C0803509F485C092
:1035A000883509F496C0883499F60E94500FD0CF20
:1035B000883909F48CC038F5883729F050F48836FA
:1035C00011F0803729F683E08093BF0210925D02EC
:1035D00057C0883809F47BC0803919F0803809F069
:1035E000B7CF80915D02803208F071C0E0915D023A
:1035F00081E08E0F80935D028091BB00F0E0E35C80
:10360000FD4F80833DC0803B39F0E0F4803A09F4FF
:1036100079C0883A09F09CCF84E08093BF02109271
:103620003C0210923B02E0917502F09176020995FE
:1036300080913B0281110FC081E080933B02109288
:103640001B0209C0803C09F4A6CF883C09F4A3CF33
:10365000883B09F07DCFE0913C0281E08E0F8093A2
:103660003C02F0E0E55EFD4F80818093BB009091CD
:103670003C0280913B0229C080919A028093BB005A
:1036800085EC8093BC0064CF9091BC028091BB021A
:10369000981758F5E091BC0281E08E0F8093BC0230
:1036A000F0E0E556FD4F8081E9CFE091BC0281E07A
:1036B0008E0F8093BC028091BB00F0E0E556FD4F79
:1036C00080839091BC028091BB029817C8F285E874
:1036D000D8CFE091BC0281E08E0F8093BC02809134
:1036E000BB00F0E0E556FD4F80838091BE02811162
:1036F0005CCF81E08093990284EA8093BC001092B1
:10370000BF0226CF85EC8093BC001092BF0280914F
:103710005D02803230F4E0915D02F0E0E35CFD4F49
:10372000108260915D0270E0E0917302F09174028A
:103730008DE392E0099510925D020ACF1092BD02CE
:1037400034CFCF93DF93E9EEF2E01382128288EE5A
:1037500093E0A0E0B0E084839583A683B78328E15B
:1037600031E03183208325EC30E03587248724EC59
:1037700030E03787268720EC30E0318B208B21EC3E
:1037800030E0338B228B22EC30E0358B248B26EC1F
:1037900030E0378B268B118E128E138E148EE6E856
:1037A000F3E01382128284839583A683B7838AE22F
:1037B00091E09183808310925904E8E3F4E0C1E042
:1037C000C083118283EC9BEAA6E7BBE382839383E9
:1037D000A483B58388ED9BE6A6E7BBE38683978346
:1037E000A087B18782EF94EEA4E6BBE3828793873C
:1037F000A487B587E8E0F4E08CE391E091838083CF
:103800008FEF9FEFDC01858B968BA78BB08F68E4E1
:1038100071E082E094E00E940E0C68E471E08CEFAD
:1038200093E00E940E0C68E471E086EF93E00E9442
:103830000E0C68E471E080EF93E00E940E0C68E4E7
:1038400071E08AEE93E00E940E0C62EB71E084EE70
:1038500093E00E940E0C69EB71E08EED93E00E9404
:103860000E0CE2E9F3E086E190E0918380838CE73F
:103870009CE8A1E0B0E084879587A687B78781EAB6
:1038800097E6A3E3BDEB808B918BA28BB38B86E68F
:1038900096E6A6EABFE3848B958BA68BB78BC0A375
:1038A00089E190E092A381A3C3A380E090E4ACE11E
:1038B000B5E484A395A3A6A3B7A310A611A612A648
:1038C00013A6AEEBB3E080E1ED0119928A95E9F71A
:1038D00014AE15AE16AE17AE1092D2031092D303EB
:1038E0001092D4031092D5031092D6031092D703EE
:1038F0001092D8031092D9031092DA031092DB03CE
:103900001092DC031092DD03DF91CF910895CF93E5
:10391000DF93CDB7DEB72C970FB6F894DEBF0FBE9E
:10392000CDBF789484B5826084BD84B5816084BD48
:1039300085B5826085BD85B5816085BD80916E004D
:10394000816080936E00109281008091810082607E
:1039500080938100809181008160809381008091BB
:1039600080008160809380008091B10084608093AA
:10397000B1008091B00081608093B00080917A00A6
:10398000846080937A0080917A00826080937A00CC
:1039900080917A00816080937A0080917A008068BB
:1039A00080937A001092C10061E08EE00E94C10312
:1039B000E091F902F091FA0282E08083E091F50251
:1039C000F091F6021082E091F702F091F8028FEC8C
:1039D000808310920103E091FD02F091FE0286E0E7
:1039E0008083E091FB02F091FC0280818061808302
:1039F000E091FB02F091FC02808188608083E0917D
:103A0000FB02F091FC02808180688083E091FB02E0
:103A1000F091FC0280818F7D808361E080E10E94D3
:103A2000C10360E080E10E94930361E08EE00E94A8
:103A3000930368EC70E080E090E00E94170484E655
:103A400090E090930201809301010E94912880935D
:103A5000670285E690E00E949128809368020091B9
:103A6000670210916802B801012E000C880B990BB7
:103A70000E9471279B01AC010E94962B811106C008
:103A80000B5011090C30110508F485C084E690E054
:103A90000E94330A68EC70E080E090E00E94170416
:103AA00061EB72E082E094E00E94690B62E074E0F6
:103AB000CE0101960E94050CCE0101960E940508D8
:103AC000CE0101960E94D10A0E94960564E670E03C
:103AD00080E090E00E94170483E0809321040E941C
:103AE000960580ED0E941408853509F47FC065EACB
:103AF00072E082E094E00E94690B1092000162E0A3
:103B000074E0CE0101960E94050CCE0101960E9440
:103B10000508CE0101960E94D10A98EE492E93E045
:103B2000592E612C712CF12CE12C2AE2C22ED12CC1
:103B30009924939480E0A82E80E0B82E68E471E088
:103B4000CE0107960E940E0C10E089EE92E00E94D2
:103B50009702181619060CF0C7C01111C5C089EEDE
:103B600092E00E9475028A3009F49FC08D3009F4FA
:103B70009CC089831A8241E050E0BE016F5F7F4F95
:103B8000CE0107960E94030B6AE070E080E090E0AF
:103B90000E941704DACF32E9E32E33E0F32E04E675
:103BA00010E0C8010E949128F70181937F010F5F07
:103BB0001F4F003B1105A9F7809192039091930349
:103BC000909304018093030164E973E0CE010196B0
:103BD0000E940E0CBE016F5F7F4F84EE93E00E9447
:103BE000860ACE0101960E94D10A54CF8AEA0E9429
:103BF000310890932304809322048CEA0E943108B8
:103C000090932504809324048EEA0E9431089093B7
:103C100027048093260480EB0E943108909333049C
:103C20008093320482EB0E94310890933504809394
:103C3000340484EB0E943108909337048093360457
:103C400086EB0E943108909329048093280488EB26
:103C50000E94310890932B0480932A048AEB0E94DF
:103C6000310890932D0480932C048CEB0E94310832
:103C700090932F0480932E048EEB0E943108909332
:103C800031048093300464EF71E080E090E00E94A2
:103C900017040E94960580E00E94F00780E10E94D0
:103CA000F00788E00E94F00738CF10916B021123D3
:103CB000C9F08B859C85892B09F466CF62EC71E095
:103CC000CE0101960E940E0CBE01695F7F4FCE01AE
:103CD00001960E94450B0E944D02CE0101960E9462
:103CE000D10A52CF11E050CFBE01695F7F4F86EFFE
:103CF00093E00E94860ACE0107960E94D10A68E4EA
:103D000071E082E094E00E94B80B8091FA039091F8
:103D1000FB038130910509F0AEC066EF73E0CE0180
:103D200001960E94050C8D819E81892B89F0E98185
:103D3000FA81309769F080818234A1F1BCF48A3233
:103D400009F496C0813439F164ED71E0833229F1D0
:103D5000BE016F5F7F4F86EF93E00E94EE0B6AE03B
:103D600070E080E090E00E94170428C0813699F04E
:103D70006CF4833469F761ED71E086EF93E00E94A3
:103D8000B80B909272028DEF9FEF16C0823651F001
:103D9000833689F3DDCF6BEC71E086EF93E00E9410
:103DA000B80B0CC06EEC71E086EF93E00E94B80B8C
:103DB000109272028CEF9FEF0E94D217CE010196F3
:103DC0000E94D10A86EF93E00E94600ACB010E9414
:103DD000D21780917202882309F43EC00E943C05EC
:103DE000A30192010E941029CA01B9010E946F2704
:103DF00020916E0230916F024091700250917102D9
:103E00000E9441292091090130910A0140910B0142
:103E100050910C010E94EF2A1816F4F40E943C0500
:103E2000A30192010E941029CA01B9010E946F27C3
:103E300060936E0270936F02809370029093710290
:103E400080916C0290916D020E94D2176AE070E03E
:103E500080E090E00E941704A114B10409F46ECE32
:103E60000E94A302882309F469CE0E94000062CE5A
:103E700067ED71E092CF049768F56AED71E0CE01CD
:103E800001960E940E0CBE016F5F7F4F86EF93E09C
:103E90000E946B0A182FCE0101960E94D10A1123AD
:103EA000C9F08091FA039091FB03029788F0E091AA
:103EB000F603F091F703309759F0818180330CF4C9
:103EC000845E9601281B310987FD3395C9017FCF98
:103ED00080E0F6CF66EF73E08CEF93E00E94EE0B8C
:103EE0000091FC031091FD030115110571F0F8011B
:103EF00081918F01882349F0082E000C990B0E94B4
:103F0000B42EF80131978083F2CF64E373E0CE01E1
:103F100001960E948E0BBE016F5F7F4F8CEF93E086
:103F20000E946B0A182FCE0101960E94D10A11231C
:103F300019F0F70109954DCF6CE273E0CE010196BF
:103F40000E948E0BBE016F5F7F4F8CEF93E00E944B
:103F50006B0A182FCE0101960E94D10A112399F104
:103F60006CED71E0CE0101960E940E0C6EED73E0D7
:103F7000CE0101960E94450BBC0182E094E00E94B4
:103F8000EE0BCE0101960E94D10A66EE71E0CE01E1
:103F900001960E940E0C62E074E0CE0101960E9430
:103FA000450BBC01CE0107960E94050CCE01079679
:103FB0000E940508CE0107960E94D10ACE01019603
:103FC0000E94D10A06CF65E273E0CE0101960E94FD
:103FD0008E0BBE016F5F7F4F8CEF93E00E946B0AE8
:103FE000182FCE0101960E94D10A112369F067E1D2
:103FF00073E082E094E00E94690B64EE73E082E07B
:1040000094E00E94620BC1CF60E173E0CE010196A3
:104010000E948E0BBE016F5F7F4F8CEF93E00E947A
:104020006B0A182FCE0101960E94D10A1123F9F0D4
:1040300047E050E066E070E0CE0101960E941F0C60
:10404000BE016F5F7F4F80EF93E00E94860ACE0132
:1040500001960E94D10A80EF93E00E94600A672BCC
:1040600019F410926B02B5CE90926B02B2CE69E059
:1040700073E0CE0101960E948E0BBE016F5F7F4FF1
:104080008CEF93E00E946B0A182FCE0101960E94DC
:10409000D10A112309F47CC04091FA035091FB032B
:1040A0004730510508F495CE66E070E0CE010196E8
:1040B0000E941F0CBE016F5F7F4F80EF93E00E9454
:1040C000860ACE0101960E94D10A8091F003909158
:1040D000F103009709F458C00E940C236093090172
:1040E00070930A0180930B0190930C016EEF72E0C4
:1040F00082E094E00E94690B4091090150910A010D
:1041000060910B0170910C0122E0CE0101960E949A
:10411000690CBE016F5F7F4FCE0107960E94050CB0
:1041200068EE71E0CE0107960E942F0BBC0182E081
:1041300094E00E94620BCE0107960E94D10ACE0144
:1041400001960E94D10A62E074E0CE0101960E94BD
:10415000050CCE0101960E940508CE0101960E9431
:10416000D10A0E943C05A30192010E941029CA01B4
:10417000B9010E946F2760936E0270936F02809363
:1041800070029093710225CE60E070E0CB01A6CF63
:1041900067EF72E0CE0101960E948E0BBE016F5F49
:1041A0007F4F8CEF93E00E946B0A182FCE0101968F
:1041B0000E94D10A112309F46AC04091FA03509178
:1041C000FB034730510508F404CE66E070E0CE01F1
:1041D00001960E941F0CBE016F5F7F4F80EF93E03E
:1041E0000E94860ACE0101960E94D10A8091F003B6
:1041F0009091F103009709F446C00E940C2360934C
:1042000005017093060180930701909308016CEEFD
:1042100072E082E094E00E94690B409105015091A8
:104220000601609107017091080121E0CE0101961D
:104230000E94690CBE016F5F7F4FCE0107960E94FE
:10424000050C68EE71E0CE0107960E942F0BBC01B1
:1042500082E094E00E94620BCE0107960E94D10A90
:10426000CE0101960E94D10A62E074E0CE0101966F
:104270000E94050CCE0101960E940508CE01019610
:104280000E94D10AA6CD60E070E0CB01B8CF67EE06
:1042900072E0CE0101960E948E0BBE016F5F7F4FD0
:1042A0008CEF93E00E946B0A182FCE0101960E94BA
:1042B000D10A112331F146E050E064E070E0CE0114
:1042C00001960E941F0CBE016F5F7F4F80EF93E04D
:1042D0000E94860ACE0101960E94D10A80EF93E0E7
:1042E0000E94600A70939303609392037093040199
:1042F0006093030180910101909102010E94330AB1
:1043000068CD63EE72E0CE0101960E948E0BBE0175
:104310006F5F7F4F8CEF93E00E946B0A182FCE01E6
:1043200001960E94D10A112309F44FC04091FA036B
:104330005091FB0363E070E0CE0101960E941F0CD8
:10434000BE016F5F7F4F80EF93E00E94860ACE012F
:1043500001960E94D10A60EF73E0CE0101960E949F
:10436000050C1F82188641E050E0BE01695F7F4F57
:10437000CE0101960E94030B811104C0CE0101966B
:104380000E94BF0ABE016F5F7F4F84EE93E00E94E0
:10439000EE0BCE0101960E94D10A0091E803109124
:1043A000E9030115110509F4A5CF01501109609128
:1043B000E4037091E503A80184E993E00E94DA2EFA
:1043C000F801EC56FC4F108295CF60EE72E0CE0102
:1043D00001960E948E0BBE016F5F7F4F8CEF93E0C2
:1043E0000E946B0A182FCE0101960E94D10A112358
:1043F00009F48AC04091FA035091FB034031510502
:1044000008F0E7CC62E070E0CE0101960E941F0C3C
:10441000BE016F5F7F4F80EF93E00E94860ACE015E
:1044200001960E94D10A8091F0039091F1030097C8
:1044300099F10E940C2320E030E048EC52E40E9405
:10444000D0270E94922A60939E0370939F038093CB
:10445000A0039093A1038B019C0100591F452140AB
:10446000310901341C4921053105D0F06AEE71E0B3
:10447000CE0101960E940E0C60EF73E0CE01019612
:104480000E94450B60EF71E00E942F0BBC0182E09F
:1044900094E00E94EE0B92CD60E070E0CB01CBCFB8
:1044A0000E94712720E030E048EC52E40E94202A6C
:1044B000AB01BC0122E0CE0101960E94690CBE0155
:1044C0006F5F7F4F82E094E00E94860ACE010196E2
:1044D0000E94D10A60E072E0CE0101960E940E0CAB
:1044E00062E074E0CE0101960E94450B6DE072E03F
:1044F0000E942F0BBC0182E094E00E94EE0BCE01E3
:1045000001960E94D10AF6CE62E172E0CE010196D8
:104510000E940E0CBE016F5F7F4F8CEF93E00E94F4
:104520006B0A182FCE0101960E94D10A112339F08F
:1045300061ED72E082E094E00E94690B95CE6DEC33
:1045400072E0CE0101960E948E0BBE016F5F7F4F1D
:104550008CEF93E00E946B0A182FCE0101960E9407
:10456000D10A112309F435CC4091FA035091FB0391
:1045700063E070E0CE0101960E941F0CBE016F5FE8
:104580007F4F80EF93E00E94860ACE0101960E9441
:10459000D10A80EF93E00E94600A70936A026093F0
:1045A000690217CC8EED93E00E94D10A84EE93E06D
:1045B0000E94D10A8AEE93E00E94D10A80EF93E034
:1045C0000E94D10A86EF93E00E94D10A8CEF93E01B
:1045D0000E94D10A82E094E00C94D10AEF920F93EA
:1045E0001F93CF93DF93E80134E047FD34E1042EBD
:1045F000000C550B57FF03C0519541955109E32E0F
:10460000022F242FAE010E94B223CE01DF91CF9161
:104610001F910F91EF900895662777270C9411252D
:104620001F93FC0199278827BC01E894119110324F
:10463000E9F3193010F01E30C8F31B3251F01D326F
:1046400049F4689406C00E946123610F711D811DA9
:10465000911D119110531A30B0F33EF4909580954E
:10466000709561957F4F8F4F9F4F1F910895FB016C
:10467000DC0105900D920020E1F70895FC01059002
:104680000020E9F7809590958E0F9F1F0895BB2716
:104690004A3031F4992322F4BDE2909581959F4FE1
:1046A0000C949923BB272A3051F4992342F4BDE29C
:1046B00090958095709561957F4F8F4F9F4F0C948B
:1046C0007723592F482F372F262F660F771F881FE4
:1046D000991F660F771F881F991F620F731F841F12
:1046E000951F660F771F881F991F0895BB27FA0132
:1046F000A62F6217710581059105330B30FB66F01B
:10470000AA27660F771F881F991FAA1FA21710F0EC
:10471000A21B63953850A9F7A05DAA3308F0A95DE4
:10472000A19336F7B111B1931082CA010C945A27A4
:10473000BB27FB015527AA27880F991FAA1FA4177B
:1047400010F0A41B83955051B9F7A05DAA3308F06F
:10475000A95DA193009779F7B111B1931192CB01A3
:104760000C945A27A9E0B0E0E8EBF3E20C94DF28C0
:104770006A01F22EB02E102FFBE3AF2EA01608F424
:104780001BE31F5F012F27E0AE014F5F5F4F0E94C9
:104790006126BC018981982F9970913009F43FC03E
:1047A0009BE2E1FC04C09E2D9170E0FC3AC05E2DBE
:1047B0005071E82FE87083FF46C084E0911101C07A
:1047C00083E0EF2DE81B8F1508F0E0E0D6018E2F77
:1047D00020E2552351F1992329F0D6019C93C6017B
:1047E00001966C0196012D5F3F4FE2FE24C08EE4DE
:1047F000D6018C9391E411969C93119712968C9309
:10480000D9018E2F90E281111BC0E20FF32FF11D11
:1048100010828EEF9FEF2996ECE00C94FB289DE22E
:10482000C6CF90E2C4CF2D9381508111FCCFCE0E24
:10483000D11CE0E0D0CF8EE6D6018C9391E6DBCFA1
:104840009D938150E0CF482F447082FF3DC084E0AB
:10485000911101C083E08F1510F4EF2DE81BD601F4
:104860008E2F20E2552309F1992329F0D6019C933C
:10487000C60101966C0196012D5F3F4FE2FE1BC001
:1048800089E4D6018C938EE411968C93119786E47B
:1048900012968C93D9018E2F90E2882309F4B5CF1C
:1048A0009D938150FACF2D9381508111FCCFCE0E74
:1048B000D11CE0E0D9CF89E6D6018C938EE6119623
:1048C0008C93119786E6E4CF9B0177FF02C030E01E
:1048D00020E0A1E0B0E0911102C0B0E0A0E0F90159
:1048E0003196AE0FBF1F8B2C912CBB2009F461C0F9
:1048F0005401EFEFAE1ABE0AAA0DBB1DFA161B0635
:1049000019F014F04F2D4A1B511188C0E3FC59C017
:104910007601A42FB0E2A1114FC0C40ED11C99237F
:1049200009F45BC040E0D6011196F60190836D0159
:10493000552309F448C0012F060F9A81582F507152
:1049400084FF03C0913309F4015010160CF047C0E6
:10495000093008F008E0EEE2FE2E5B01A01AB10873
:1049600085019194819491082F3F320729F4D60153
:10497000FC92F60131966F016217730794F10217EA
:1049800013077CF5DB01A21BB30BAA24A394B12C63
:10499000AC0EBD1EAA0DBB1D11968C912150310984
:1049A000D601119628153905F4F0F60180836D01C2
:1049B000DBCFB12CA12CA0CFF701B1937F01A15087
:1049C000AACF9111B0CFD601942F50E302C05D93CE
:1049D00091509111FCCFC40ED11C40E0ACCF01E04E
:1049E000BACF80E3DBCF6217730731F4963388F4D4
:1049F000953311F4552369F0F6018083FD01842F6E
:104A000090E2811108C0A40FB11D1C9290E080E0DB
:104A100002CF81E3F1CF91938150F3CF911183CFF6
:104A20008ACFB0E0A0E0E7E1F5E20C94DF285C017A
:104A30007B016115710519F0DB018D939C93850154
:104A40000F5F1F4FF501D0818D2F90E00E94392715
:104A50006C01892BB9F5DD32B9F50F5F1F4FD50118
:104A60001196DC91C1E05801F1E0AF1AB10843E0C2
:104A700050E060E271E0C5010E944227892B69F590
:104A8000680182E0C80ED11C45E050E06BE171E0A6
:104A9000C6010E944227892B21F4680197E0C90EC4
:104AA000D11CE114F10419F0D701CD92DC9260E041
:104AB00070E080E89FEFC111FFC060E070E080E827
:104AC0009FE7FAC05801BBCFDB3229F485010E5FA6
:104AD0001F4FF501D181C0E0C6CF43E050E068E14F
:104AE00071E0C5010E944227892BE9F0F80110E02E
:104AF00000E020E030E0A9015F01B0ED8B2E8D0ECB
:104B000089E08815C8F19C2E689491F88C2F8870E4
:104B1000C2FF16C0811102C00F5F1F4F3196D50131
:104B2000DC91C92DE9CFE114F10429F00E5F1F4F8C
:104B3000F7011183008360E070E080EC9FE7BCC068
:104B4000882311F001501109A5E0B0E00E94C628A9
:104B50009B01AC01220F331F441F551F280D311D2F
:104B6000411D511D283999E93907490799E159072C
:104B7000A8F2C6609C2ED2CFAEEF8A1206C0C3FD4B
:104B80003CC09C2E689493F8C9CFDF7DD534A9F53D
:104B900080818D3239F4C061DF011296818162E03B
:104BA00070E006C0DF018B32C1F3119661E070E066
:104BB00080535D01A61AB70A8A30F8F4E0E8CE16F1
:104BC000ECE0DE065CF4B601660F771F660F771F18
:104BD000C60ED71ECC0CDD1CC80ED11C5D01FFEF2C
:104BE000AF1ABF0A8C9180538A30A8F1C4FF03C06A
:104BF000D194C194D1080C0D1D1DC1FF09C0E11451
:104C0000F10431F081E0A81AB108D701AD92BC924D
:104C1000CA01B9010E946F27C370C33009F49058CC
:104C20004B015C0120E030E0A9010E946A27882343
:104C300009F440C0CFE4D1E017FF05C011950195FC
:104C40001109C7E3D1E06E01B8E1CB1AD10880E2C7
:104C5000E82EF12C0FC0D501B1CFFE012591359181
:104C6000459154910E191F09C501B4010E94D02726
:104C70004B015C01D501C4010E151F0574F7249783
:104C8000F594E794CC16DD06A9F78A2F880F8B2FB1
:104C9000881F8F3F49F020E030E0A901C501B40131
:104CA0000E946A27811106C082E290E090935B0423
:104CB00080935A04C501B401CDB7DEB7ECE00C9483
:104CC000FB28283008F027E03327DA01990F311D3F
:104CD00087FD916000966105710539F432602E5FA1
:104CE0003D9330E32A95E1F708959F3F30F08038F7
:104CF0007105610509F03C5F3C5F3D93913008F020
:104D00008068911DDF93CF931F930F93FF92EF92D3
:104D1000192F987F9695E92F96959695E90FFF277D
:104D2000E355FE4F99273327EE24FF24A701E7011F
:104D300005900894079428F4360FE71EF81E491FC3
:104D4000511D660F771F881F991F0694A1F70590C4
:104D5000079428F4E70EF81E491F561FC11D770F50
:104D6000881F991F661F0694A1F70590079428F4E1
:104D7000F80E491F561FC71FD11D880F991F661FA8
:104D8000771F0694A1F70590079420F4490F561F4A
:104D9000C71FD81F990F661F771F881F0694A9F792
:104DA00084911095177041F0D695C7955795479502
:104DB000F794E7941A95C1F7E3E5F1E0689415904C
:104DC000159135916591959105907FE27395E11864
:104DD000F10A430B560BC90BD009C0F7E10CF11EC9
:104DE000431F561FC91FD01D7EF4703311F48A95DE
:104DF000E6CFE894015030F0080F0AF400270217BC
:104E000008F4202F2395022F7A3328F079E37D933D
:104E10002A95E9F710C07D932A9589F6069497950F
:104E20006795379517951794E118F10A430B560BC0
:104E3000C90BD00998F023957E9173957A3308F0C9
:104E400070E37C932013B8F77E9170617D9330F00E
:104E5000839571E37D9370E32A95E1F71124EF9038
:104E6000FF900F911F91CF91DF91992787FD90952A
:104E7000089591110C943D28803219F08950855085
:104E8000C8F70895FB01DC014150504088F08D9136
:104E900081341CF08B350CF4805E659161341CF01C
:104EA0006B350CF4605E861B611171F3990B0895EC
:104EB000881BFCCFDC01FC01672F71917723E1F7A0
:104EC000329704C07C916D9370836291AE17BF07D7
:104ED000C8F308950E94AC2708F481E00895E8948F
:104EE00009C097FB3EF490958095709561957F4F32
:104EF0008F4F9F4F9923A9F0F92F96E9BB279395E0
:104F0000F695879577956795B795F111F8CFFAF4EF
:104F1000BB0F11F460FF1BC06F5F7F4F8F4F9F4F20
:104F200016C0882311F096E911C0772321F09EE87E
:104F3000872F762F05C0662371F096E8862F70E0E4
:104F400060E02AF09A95660F771F881FDAF7880FBE
:104F50009695879597F90895990F0008550FAA0B14
:104F6000E0E8FEEF16161706E807F907C0F012167C
:104F70001306E407F50798F0621B730B840B950B7F
:104F800039F40A2661F0232B242B252B21F40895D4
:104F90000A2609F4A140A6958FEF811D811D089571
:104FA0000E94E3270C9457280E94492838F00E9459
:104FB000502820F0952311F00C9440280C9446289A
:104FC00011240C948B280E94682870F3959FC1F3DC
:104FD000950F50E0551F629FF001729FBB27F00DA7
:104FE000B11D639FAA27F00DB11DAA1F649F6627FC
:104FF000B00DA11D661F829F2227B00DA11D621F4B
:10500000739FB00DA11D621F839FA00D611D221F04
:10501000749F3327A00D611D231F849F600D211DE8
:10502000822F762F6A2F11249F5750409AF0F1F06B
:1050300088234AF0EE0FFF1FBB1F661F771F881FD4
:1050400091505040A9F79E3F510580F00C944028A4
:105050000C948B285F3FE4F3983ED4F386957795C4
:105060006795B795F795E7959F5FC1F7FE2B880F7A
:10507000911D9695879597F9089599278827089502
:1050800097F99F6780E870E060E008959FEF80ECFB
:10509000089500240A94161617061806090608959E
:1050A00000240A9412161306140605060895092E04
:1050B0000394000C11F4882352F0BB0F40F4BF2B73
:1050C00011F460FF04C06F5F7F4F8F4F9F4F0895B3
:1050D00057FD9058440F551F59F05F3F71F04795A9
:1050E000880F97FB991F61F09F3F79F0879508958E
:1050F000121613061406551FF2CF4695F1DF08C0AD
:10510000161617061806991FF1CF869571056105C9
:1051100008940895E894BB2766277727CB0197F971
:105120000895F999FECF92BD81BDF89A992780B56F
:105130000895262FF999FECF1FBA92BD81BD20BDDB
:105140000FB6F894FA9AF99A0FBE01960895052EB3
:1051500097FB1EF400940E94BE2857FD07D00E94C2
:10516000102907FC03D04EF40C94BE2850954095AE
:10517000309521953F4F4F4F5F4F08959095809503
:10518000709561957F4F8F4F9F4F08950E943229F0
:10519000A59F900DB49F900DA49F800D911D11248B
:1051A0000895B7FF0C94C6280E94C628821B930B53
:1051B00008952F923F924F925F926F927F928F92BB
:1051C0009F92AF92BF92CF92DF92EF92FF920F9396
:1051D0001F93CF93DF93CDB7DEB7CA1BDB0B0FB6A0
:1051E000F894DEBF0FBECDBF09942A88398848885D
:1051F0005F846E847D848C849B84AA84B984C884F3
:10520000DF80EE80FD800C811B81AA81B981CE0FE9
:10521000D11D0FB6F894DEBF0FBECDBFED010895CE
:10522000A1E21A2EAA1BBB1BFD010DC0AA1FBB1FAA
:10523000EE1FFF1FA217B307E407F50720F0A21B1C
:10524000B30BE40BF50B661F771F881F991F1A9489
:1052500069F760957095809590959B01AC01BD01B3
:10526000CF010895A29FB001B39FC001A39F700D0D
:10527000811D1124911DB29F700D811D1124911D5E
:1052800008955058BB27AA270E9459290C945728E3
:105290000E94492838F00E94502820F039F49F3F9E
:1052A00019F426F40C9446280EF4E095E7FB0C94D0
:1052B0004028E92F0E94682858F3BA17620773073D
:1052C0008407950720F079F4A6F50C948A280EF44B
:1052D000E0950B2EBA2FA02D0B01B90190010C0106
:1052E000CA01A0011124FF27591B99F0593F50F41E
:1052F000503E68F11A16F040A22F232F342F442776
:10530000585FF3CF469537952795A795F04053956D
:10531000C9F77EF41F16BA0B620B730B840BBAF03D
:105320009150A1F0FF0FBB1F661F771F881FC2F7A8
:105330000EC0BA0F621F731F841F48F487957795BC
:105340006795B795F7959E3F08F0B0CF9395880F76
:1053500008F09927EE0F9795879508950E944928A0
:1053600060F080E891E009F49EEF0E94502828F058
:1053700040E851E071F45EEF0CC00C9446280C94A8
:105380008A28E92FE0780E94682840F3092E052A30
:10539000B1F3261737074807590738F00E2E07F8DC
:1053A000E02569F0E025E0640AC0EF6307F80094A7
:1053B00007FADB01B9019D01DC01CA01AD01EF93E0
:1053C0000E94372A0E9457280E94F1295F91552395
:1053D00039F02BED3FE049E450FD49EC0C944229B3
:1053E0000895DF93DD27B92FBF7740E85FE31616F6
:1053F000170648075B0718F4D92F0E94F42A9F93D9
:105400008F937F936F930E94922BE8E6F0E00E94C7
:10541000C82A0E9457282F913F914F915F910E9477
:10542000E327DD2351F09058A2EA2AED3FE049EC52
:105430005FE3D0785D270E945929DF910C945728AB
:105440000E94342A0C9457280E94502858F00E9439
:10545000492840F029F45F3F29F00C94402851116D
:105460000C948B280C9446280E94682868F3992392
:10547000B1F3552391F3951B550BBB27AA27621750
:105480007307840738F09F5F5F4F220F331F441F5D
:10549000AA1FA9F335D00E2E3AF0E0E832D0915091
:1054A0005040E695001CCAF72BD0FE2F29D0660F7E
:1054B000771F881FBB1F261737074807AB07B0E8C1
:1054C00009F0BB0B802DBF01FF2793585F4F3AF0C7
:1054D0009E3F510578F00C9440280C948B285F3F38
:1054E000E4F3983ED4F3869577956795B795F7954D
:1054F0009F5FC9F7880F911D9695879597F9089535
:10550000E1E0660F771F881FBB1F621773078407D0
:10551000BA0720F0621B730B840BBA0BEE1F88F7DF
:10552000E09508950E94992A6894B1110C948B28F3
:1055300008950E94702888F09F5798F0B92F9927F6
:10554000B751B0F0E1F0660F771F881F991F1AF06E
:10555000BA95C9F714C0B13091F00E948A28B1E021
:1055600008950C948A28672F782F8827B85F39F020
:10557000B93FCCF3869577956795B395D9F73EF407
:1055800090958095709561957F4F8F4F9F4F0895AF
:10559000DF93CF931F930F93FF92EF92DF927B01E4
:1055A0008C01689406C0DA2EEF010E94E327FE0109
:1055B000E894A5912591359145915591A6F3EF0178
:1055C0000E945929FE019701A801DA9469F7DF903A
:1055D000EF90FF900F911F91CF91DF9108950E945E
:1055E000AC2708F48FEF08959B01AC0160E070E0F8
:1055F00080E89FE30C94202AFA01EE0FFF1F3096FB
:1056000021053105A1F16115710561F48038BFE311
:105610009B0749F168949038810561F08038BFEFAD
:105620009B0741F099234AF5FF3FE105310521052C
:1056300019F1E8940894E795D901AA2329F4AB2F2E
:10564000BE2FF85FD0F310C0FF5F70F4A695E0F7AF
:10565000F73950F019F0FF3A38F49F779F930DD047
:105660000F9007FC9058089546F00C94462860E08F
:1056700070E080E89FE308954FE79F775F934F9333
:105680003F932F930E942C2C2F913F914F915F912C
:105690000E94D0270C94A32B19F416F40C944628DE
:1056A0000C94D52B0E947028B8F39923C9F3B6F354
:1056B0009F57550B87FF0E94E32B0024A0E640EA8A
:1056C000900180585695979528F4805C660F771F57
:1056D000881F20F026173707480730F4621B730B2A
:1056E000840B202931294A2BA6951794079420254D
:1056F00031254A2758F7660F771F881F20F0261795
:105700003707480730F4620B730B840B200D311DF3
:10571000411DA09581F7B901842F9158880F969566
:10572000879508959B01AC010C94D0270E94AC276B
:10573000880B990B089529F416F00C9440280C94CA
:105740008A280C9446280E947028A8F39638A0F75F
:1057500007F80F92E8942BE33AEA48EB5FE70E94E0
:10576000E6270F920F920F924DB75EB70F920E94ED
:10577000742CE5E9F0E00E94C82A4F915F91EF9107
:10578000FF91E595EE1FFF1F49F0FE57E0684427A3
:10579000EE0F441FFA95E1F74195550B0E94EE2B51
:1057A0000F9007FE0C94F42A08959F3F31F091501A
:1057B00020F4879577956795B795880F911D9695F5
:1057C000879597F9089591505040660F771F881F6D
:1057D000D2F708950C9440280C94D52B0E94702881
:1057E000D8F39923C9F3940F511DA3F3915050405E
:1057F00094F059F0882332F0660F771F881F91507C
:105800005040C1F79E3F51052CF7880F911D96958A
:10581000879597F908955F3FACF0983E9CF0BB27C1
:10582000869577956795B79508F4B1609395C1F71C
:10583000BB0F58F711F460FFE8CF6F5F7F4F8F4FBA
:105840009F4FE3CF0C948B2816F00C94D52B0C941F
:10585000462868940C9440280E947028A8F3992345
:10586000C1F3AEF3DF93CF931F930F93FF92C92F32
:10587000DD2788232AF02197660F771F881FDAF724
:1058800020E030E040E85FEB9FE3883920F0803E85
:1058900038F021968F770E944229EDEBF0E004C0AA
:1058A0000E944229EAEEF0E00E94C82A8B01BE0164
:1058B000EC01FB2E6F5771097595771F880B990BBB
:1058C0000E94712728E132E741E35FE30E94E3276A
:1058D000AF2D9801AE01FF900F911F91CF91DF91F5
:1058E0000E9459290C945728FA01DC01AA0FBB1F0A
:1058F0009B01AC01BF5728F4222733274427507857
:1059000020C0B75190F4AB2F0024469537952795CA
:10591000011CA395D2F3002071F0220F331F441F06
:10592000B395DAF30ED00C94412961307105A0E8EB
:105930008A07B94630F49B01AC0166277727882790
:105940009078309621F020833183428353830895E9
:10595000DB018F939F930E94C628BF91AF91A29FB6
:10596000800D911DA39F900DB29F900D112408955D
:10597000AA1BBB1B51E107C0AA1FBB1FA617B70775
:1059800010F0A61BB70B881F991F5A95A9F7809591
:105990009095BC01CD010895EE0FFF1F0590F49185
:1059A000E02D09940F931F93CF93DF9382309105DD
:1059B00010F482E090E0E0915E04F0915F0430E04A
:1059C00020E0B0E0A0E0309799F42115310509F40A
:1059D0004AC0281B390B24303105D8F58A819B81B8
:1059E0006115710589F1FB0193838283FE0111C06A
:1059F000408151810281138148175907E0F048170F
:105A0000590799F4109761F012960C931297139618
:105A10001C933296CF01DF91CF911F910F91089582
:105A200000935E0410935F04F4CF2115310551F00B
:105A30004217530738F0A901DB019A01BD01DF01CC
:105A4000F801C1CFEF01F9CF90935F0480935E041A
:105A5000CDCFFE01E20FF31F8193919322503109C4
:105A600039832883D7CF20915C0430915D04232BA8
:105A700041F4209110013091110130935D04209385
:105A80005C0420910E0130910F012115310541F484
:105A90002DB73EB74091120150911301241B350BD5
:105AA000E0915C04F0915D04E217F307A0F42E1B73
:105AB0003F0B2817390778F0AC014E5F5F4F241772
:105AC000350748F04E0F5F1F50935D0440935C0410
:105AD000819391939FCFF0E0E0E09CCFCF93DF9351
:105AE0000097E9F0FC01329713821282A0915E04C4
:105AF000B0915F04ED0130E020E01097A1F4208127
:105B00003181820F931F20915C0430915D0428172E
:105B1000390709F061C0F0935D04E0935C04DF9104
:105B2000CF910895EA01CE17DF07E8F54A815B813E
:105B30009E0141155105B1F7E901FB83EA834991C3
:105B40005991C40FD51FEC17FD0761F48081918135
:105B50000296840F951FE90199838883828193813E
:105B60009B838A83F0E0E0E012968D919C911397DD
:105B70000097B9F52D913C911197CD010296820FB6
:105B8000931F20915C0430915D042817390739F682
:105B9000309751F510925F0410925E04B0935D044B
:105BA000A0935C04BCCFD383C28340815181840F16
:105BB000951FC817D90761F44E5F5F4F888199819F
:105BC000480F591F518340838A819B81938382832D
:105BD0002115310509F0B0CFF0935F04E0935E0426
:105BE0009ECFFD01DC01C0CF13821282D7CFB0E07F
:105BF000A0E0EDEFFDE20C94DB288C01009751F45E
:105C0000CB010E94D22C8C01C801CDB7DEB7E0E1F8
:105C10000C94F728FC01E60FF71F9C012250310974
:105C2000E217F30708F49DC0D901CD91DC911197DB
:105C3000C617D70798F0C530D10530F3CE010497C9
:105C40008617970708F3C61BD70B2297C193D193EA
:105C50006D937C93CF010E946E2DD6CF5B01AC1A61
:105C6000BD0A4C018C0E9D1EA0915E04B0915F0494
:105C7000512C412CF12CE12C109731F580915C04D2
:105C800090915D048815990509F05CC04616570689
:105C900008F058C080910E0190910F01009741F4D7
:105CA0008DB79EB74091120150911301841B950B43
:105CB000E817F90708F055C0F0935D04E0935C0421
:105CC000F90171836083A0CF8D919C9111971296F9
:105CD0006C90129713967C901397A815B90559F5F7
:105CE0006C0142E0C40ED11CCA14DB0420F1AC01EB
:105CF0004A195B09DA011296159780F06282738265
:105D000051834083D9016D937C93E114F10471F0C8
:105D1000D7011396FC93EE93129776CF22968C0FB1
:105D20009D1FF90191838083F301EFCFF0935F040E
:105D3000E0935E0469CF4816590608F42C017D01F2
:105D4000D3019ACFCB010E94D22C7C01009749F05D
:105D5000AE01B8010E94BC2EC8010E946E2D8701C1
:105D600053CF10E000E050CF9111089581568A5131
:105D700008F4805285580895FB01DC0102C00190AF
:105D80000D9241505040D8F70895FB01DC0101907D
:105D90000D920020E1F70895FB01DC0141505040D5
:105DA00030F08D910190801919F40020B9F7881B0B
:105DB000990B0895FB01DC014150504048F00190DF
:105DC0000D920020C9F701C01D9241505040E0F7EC
:105DD000089511E0C2ECD1E004C0FE010E94CC2C79
:105DE0002196C33CD107C9F7F894FFCF0164001690
:105DF000000000A0400000F04101000060048000AD
:105E000000000000D90220026602260397027502F4
:105E1000890200000000C1079407020884074905B1
:105E2000ED018507000000004805D90A5005850EE0
:105E3000380E0D0A00543D006F432000483D0025F8
:105E400000484D433538383300436F6D70617373CC
:105E50003A2000286465672920004E200045005341
:105E600020005700732000296D4700203D3E000AA6
:105E70003E006F4320413D006D00613D0020670002
:105E8000496E636C2E20616E672E28782079207A07
:105E9000292F6465673A2000613A00672000414E6F
:105EA0004D4C3033004E616E6F413262330073658A
:105EB0007269616C3A20002D35002D34002D3300BD
:105EC0002D32002D3100440056657273696F6E3AB1
:105ED000200023007300534C20503D005061206986
:105EE0007320756E6C696B656C7921005365612058
:105EF0006C6576656C20503D0020685061005556F9
:025F00005A0045
:107E0000112484B714BE81FFF0D085E080938100F7
:107E100082E08093C00088E18093C10086E0809377
:107E2000C20080E18093C4008EE0C9D0259A86E02C
:107E300020E33CEF91E0309385002093840096BBD3
:107E4000B09BFECF1D9AA8958150A9F7CC24DD24C4
:107E500088248394B5E0AB2EA1E19A2EF3E0BF2EE7
:107E6000A2D0813461F49FD0082FAFD0023811F036
:107E7000013811F484E001C083E08DD089C08234E0
:107E800011F484E103C0853419F485E0A6D080C0E4
:107E9000853579F488D0E82EFF2485D0082F10E0AE
:107EA000102F00270E291F29000F111F8ED06801E7
:107EB0006FC0863521F484E090D080E0DECF843638
:107EC00009F040C070D06FD0082F6DD080E0C81688
:107ED00080E7D80618F4F601B7BEE895C0E0D1E017
:107EE00062D089930C17E1F7F0E0CF16F0E7DF06D8
:107EF00018F0F601B7BEE89568D007B600FCFDCFD4
:107F0000A601A0E0B1E02C9130E011968C91119780
:107F100090E0982F8827822B932B1296FA010C0160
:107F200087BEE89511244E5F5F4FF1E0A038BF0790
:107F300051F7F601A7BEE89507B600FCFDCF97BE46
:107F4000E89526C08437B1F42ED02DD0F82E2BD052
:107F50003CD0F601EF2C8F010F5F1F4F84911BD097
:107F6000EA94F801C1F70894C11CD11CFA94CF0C13
:107F7000D11C0EC0853739F428D08EE10CD085E9AC
:107F80000AD08FE07ACF813511F488E018D01DD067
:107F900080E101D065CF982F8091C00085FFFCCF94
:107FA0009093C60008958091C00087FFFCCF809118
:107FB000C00084FD01C0A8958091C6000895E0E648
:107FC000F0E098E1908380830895EDDF803219F02E
:107FD00088E0F5DFFFCF84E1DECF1F93182FE3DFCA
:107FE0001150E9F7F2DF1F91089580E0E8DFEE27F6
:047FF000FF270994CA
:027FFE00040479
:00000001FF
